:0200000480007A
:100000009710000093800000171100001301810178
:1000100083A1000013020000930210001303F0FFFD
:10002000B70300809383F3FF37040080930F000031
:100030006384410093EF1F006384510093EF2F000E
:100040006384610093EF4F006384710093EF8F002E
:100050006384810093EF0F012320310023224100AC
:10006000232451002326610023287100232A8100C4
:10007000232CF10197100000938000F91711000064
:10008000130101FC03A300009303000013041000FC
:100090009304F0FF370500801305F5FFB7050080D6
:1000A000930F00006304730093EF1F006304830049
:1000B00093EF2F006304930093EF4F006304A300BA
:1000C00093EF8F006304B30093EF0F0123206100CF
:1000D0002322710023248100232691002328A100DC
:1000E000232AB100232CF10197100000938000F225
:1000F00017110000130181F603A60000930600000B
:10010000130710009307F0FF370800801308F8FF6B
:10011000B7080080930F00006304D60093EF1F0020
:100120006304E60093EF2F006304F60093EF4F00A3
:100130006304060193EF8F006304160193EF0F0130
:100140002320C1002322D1002324E1002326F10033
:1001500023280101232A1101232CF101971000000B
:10016000938000EB17110000130101F103A90000B7
:1001700093090000130A1000930AF0FF370B008068
:10018000130BFBFFB70B0080930F000063043901D2
:1001900093EF1F006304490193EF2F00630459019B
:1001A00093EF4F006304690193EF8F0063047901BB
:1001B00093EF0F0123202101232231012324410148
:1001C0002326510123286101232A7101232CF101E7
:1001D00097100000938000E417110000130181EBD9
:1001E00003AC0000930C0000130D1000930DF0FF02
:1001F000370E0080130EFEFFB70E0080930F000035
:1002000063049C0193EF1F006304AC0193EF2F0084
:100210006304BC0193EF4F006304CC0193EF8F00A4
:100220006304DC0193EF0F0123208101232291015C
:100230002324A1012326B1012328C101232AD101AE
:10024000232CF101971D0000938D8DE69300000093
:10025000130110009301F0FF370200801302F2FF38
:10026000B7020080930F00006384000093EF1F002B
:100270006304010093EF2F006384010093EF4F00AC
:100280006304020093EF8F006384020093EF0F0179
:100290006304100093EF0F026304200093EF0F0438
:1002A0006304300093EF0F086304400093EF0F10D6
:1002B0006304500093EF0F2023A0FD01971A000064
:1002C000938A8AD5171B0000130BCBDE83AF0A007D
:1002D0001301F0FF9301F0FF37D2ED0F130292BA32
:1002E00063840F0213010000930100001302000059
:1002F000B74165879381113263840F0213010000B7
:10030000930100001302000037E1BC9A130101EFD2
:10031000E3800FFE130100009301000013020000B0
:1003200023200B0023222B0023243B0023264B00F9
:1003300017150000130505CF97150000938585D884
:10034000370610F01306C6F26306B5028326C50011
:100350002320D600832685002320D600832645004F
:100360002320D600832605002320D600130505018F
:100370006FF09FFD370510F0130505F223200500EF
:040380000000000079
:101000000000000001000000FFFFFFFFFFFFFF7F67
:101010000000008000000000000000000000000050
:10102000FFFFFFFFFFFFFFFFFFFFFFFFFFFFFFFFD0
:10103000FFFFFFFFFFFFFFFFFFFFFFFFFFFFFFFFC0
:10104000FFFFFFFFFFFFFFFFFFFFFFFFFFFFFFFFB0
:10105000FFFFFFFFFFFFFFFFFFFFFFFFFFFFFFFFA0
:10106000FFFFFFFFFFFFFFFFFFFFFFFFFFFFFFFF90
:10107000FFFFFFFFFFFFFFFFFFFFFFFFFFFFFFFF80
:10108000FFFFFFFFFFFFFFFFFFFFFFFFFFFFFFFF70
:10109000FFFFFFFFFFFFFFFFFFFFFFFFFFFFFFFF60
:1010A000FFFFFFFFFFFFFFFFFFFFFFFFFFFFFFFF50
:1010B000FFFFFFFFFFFFFFFFFFFFFFFFFFFFFFFF40
:040000058000000077
:00000001FF
